:10367400000A0014000500320032000A0005000AA6
:02368400C35031
:1031C400C10B4101770101BE010156000149000113
:1031D4005A00015B00014700014B00014C00C10A89
:1031E400C1000145FF41011F0041015400015E007F
:0E31F400C103C182C108014A00015D00C10192
:10280000E4F524F525F5A0F590F5D8121A9BE4908F
:10281000011FF01217E11234DF300926C209786E69
:10282000E6600B16E6B4010620050312354CE5629E
:10283000D39400400DD5620A1236B97F0A7E001289
:1028400036AE78A3E6D394034050E4F61236CF12A6
:102850003000E4F55CE55C25E024ACF8E6FE08E633
:10286000FF900178EEF0A3EFF04E6025E024FFF03A
:10287000900178E034FFF0E0FEA3E0FFE55C25E0A6
:1028800024ACF8A60608A607EF4E7005AF5C12361A
:1028900062055CE55CC3940940BBE5567002011912
:1028A0001556744D2556F8E614602614602D1470E4
:1028B00002213424FC7002213E240770DD0525E549
:1028C00025C3940A4005E4F525B204E4FDFCFF802D
:1028D000681208EDE4FDFC7F01805EE51C700312C8
:1028E00034DF301521C215E4F5249000FDE0FF121D
:1028F000000040397F057E001236AE0524E524C372
:10290000940540E68027301421C214E4F524900099
:10291000FBE0FF12000040157F057E001236AE0579
:1029200024E524C3940540E68003122BB0E4FDFCAB
:102930007F028005E4FDFC7F031234AA019AE4FFC4
:082940001218001234A5019ADF
:101A9B00E4F580123686900050741EF0E490018AB3
:101AAB00F090018AE0FFC394205052EF244EFF7B4D
:101ABB00017A01798CE4F533122D96401190018A4D
:101ACB00E02492F582E43400F583E4F08027D39090
:101ADB00018DE0940590018CE094004004E4F0A3A8
:101AEB00F090018DE0FF90018AE02492F582E434BE
:101AFB0000F583EFF090018AE004F080A43000122F
:101B0B00D2A0D2A1D2A2D2A3D2A4D2A5D2A6D2A71E
:101B1B008010C2A0C2A1C2A2C2A3C2A4C2A5C2A667
:101B2B00C2A7D2B4D294D295C2B7C2B5C2B6C29331
:101B3B00C297C2B37B017A01798BE4F5347F0F1224
:101B4B003136400690018B7401F090018BE0B401AB
:101B5B000B7587809000FC7403F08009E4F5879087
:101B6B0000FC7406F07580FF759850758921758D92
:101B7B00FD758BFD758A04758CF7D28ED28CD2A92C
:101B8B0043BF021232C1D2AFD2AC7548011236CF6D
:101B9B001236AA1236CF1236AA1236CF1236AA1224
:101BAB0036CF1236AA1236CF1236AA1236CFE4F53A
:101BBB004890018AF090018AE0FFC3941A5018EF05
:101BCB0025E02420F582E43401F583E4F0A3F090C2
:101BDB00018AE004F080DEE490018AF090018AE053
:101BEB00FFC39408500B74A42FF8E4F6E004F080C4
:101BFB00EBE490018AF090018AE0FFC39409500F47
:101C0B00EF25E024ACF8E4F608F6E004F080E7E416
:101C1B00FBFDFC7F63120F94E490011EF07B017AB5
:101C2B00017975F5347F0D123136400690017574CC
:101C3B0080F07B017A017977E4F5347F0C12313631
:101C4B00400AE4FB7D01FC7F0C120F94900177E0BE
:101C5B00700FFB7D01FC7F0C120F949001777401C8
:101C6B00F0E4FB7D0DFC7F05120F94E4FB7D15FC6E
:101C7B007F07120F947B017A01791FE4F5347F08FB
:101C8B00123136E4FDFCFF1234AAE4FDFC7F021294
:101C9B0034AAE4FDFC7F011234AA1234A59001771B
:101CAB00E06402703BFDFC7F041234AAE490018ACD
:101CBB00F090018AE0FFC394105018EF25E02455F3
:101CCB00F582E43401F583E4F0A3F090018AE0049B
:101CDB00F080DE90011EE030E704D2068002C206DF
:101CEB00E4FDFC7F081234AAE490018AF090018A8B
:101CFB00E0FFC39420501474722FF582E43400F586
:0B1D0B0083E4F090018AE004F080E225
:011D160022AA
:03000B00021F8F42
:101F8F00C0E0C0F0C083C082C0D075D000C000C018
:101F9F0001C002C003C004C005C006C007758A0493
:101FAF00758CF778A306D2097580FF78BE06E6D345
:101FBF00940340027601123357D007D006D005D0D4
:101FCF0004D003D002D001D000D0D0D082D083D0A3
:041FDF00F0D0E0322C
:10366200E556C39409500AAE560556744D2EF8A677
:0236720007222D
:0534A500E4FDFC7F07BF
:1034AA008C268D27E5274526701FEF25E02474F525
:1034BA0082E43436F583E493FC740193FDEF25E04E
:1034CA0024ACF8A60408A60522EF25E024ACF8A649
:0534DA002608A62722D0
:1017E10090011FE0FF7006439B4075A303EFC39474
:0E17F100014002D20AEFC394034002D200224C
:102BB000200A02D2B2E51CB40109D20C7F08122C03
:102BC000BD8012E51CB40205122E4D8008E51CB430
:102BD0000303122A8720080281BC300A67E4F52625
:102BE000E52625E02420F582E43401F583E0FEA308
:102BF000E0FFD39464EE94005019E52625E02430DC
:102C0000F582E43401F583E0FCA3E0D39464EC9412
:102C1000004022C3EF9484EE9403401FE52625E094
:102C20002430F582E43401F583E0FEA3E0C394840C
:102C3000EE94034006900154E004F00526E526B426
:102C4000089E8068E4F526E52625E02430F582E438
:102C50003401F583E0FEA3E0FFE52625E02420F51E
:102C600082E43401F583E0FCA3E0C39FFFEC9EFE09
:102C7000123698D3EF9432EE648094804025900110
:102C800054E004F074079526FFE55EA8070880036A
:102C9000A2E713D8FB4401FEA807088002C333D87B
:102CA000FCF55E0526E526C39408409B900154E0A0
:0C2CB000B4FF05C202C20822D202C20812
:012CBC0022F5
:021800008F2631
:10180200E4F52AD20FE5261460390470798580291F
:10181200A2B7920CA2B5920DA2B6920EC2B7C2B5F1
:10182200C2B67580FFC2B47F0A7E001236AEC29481
:10183200858027D2947580FFC295858028D295D263
:10184200B48034858029A2B7920CA2B5920DA2B6BB
:10185200920EC2B7C2B5C2B67580FFC2107F0A7EB1
:10186200001236AEC294858027D2947580FFC2954D
:10187200858028D295D210852980A20C92B7A20D1C
:1018820092B5A20E92B67D01E4FCE5275D7003D30A
:101892008001C3500AE5285D70028001C34003ED58
:1018A200422AED25E0FD0CBC08E0745B2526F8E633
:1018B200652A6023744C2526F806744C2526F8E622
:1018C200C3940A4019745B2526F8A62A744C25266F
:1018D200F8E4F6D20F8007744C2526F8E4F6744932
:1018E2002526F8E66527602374472526F8067447FF
:1018F2002526F8E6C3940A401974492526F8A62736
:1019020074472526F8E4F6D20F800774472526F897
:10191200E4F6745A2526F8E665286023744B2526DA
:10192200F806744B2526F8E6C3940A4019745A2522
:1019320026F8A628744B2526F8E4F6D20F80077401
:101942004B2526F8E4F67D01200F02413DC20FE54A
:10195200267074FC745B2526F8E65D7002802274A2
:10196200492526F8E65D700874A42CF876018017E4
:10197200745A2526F8E65D700874A42CF876028065
:101982000674A42CF8E4F6ED25E0FD0CBC08C5E4D1
:10199200900140F0A3F0FC900140E0FEA3E0780249
:1019A200C333CE33CED8F9FF900140EEF0A3EFF06F
:1019B20074A42CF8E6FBEB4FFF900140EEF0A3EF8E
:1019C200F00CBC08D280747C08745B2526F8E65DB6
:1019D2007002802274492526F8E65D700874A42CF2
:1019E200F876018017745A2526F8E65D700874A40B
:1019F2002CF87602800674A42CF8E4F6ED25E0FDBE
:101A02000CBC10C5E4900142F0A3F07C08900142A6
:101A1200E0FEA3E07802C333CE33CED8F9FF9001C3
:101A220042EEF0A3EFF074A42CF8E6FBEB4FFF902C
:101A32000142EEF0A3EFF00CBC10D2900177E0FF70
:101A42007048E5267023900140E0FAA3E0FB4A606B
:101A520010EB64AA7003EA64AA6006BA5507BB5584
:101A620004D2038025C2038021900142E0FAA3E060
:101A7200FB4A6010EB64AA7003EA64AA6006BA55D6
:101A820007BB5504D2038002C203EFB4030A7C08E9
:081A920078A47402F608DCFCE4
:011A9A002229
:10300000900177E070123004055358FE8003435856
:103010000130031D801680193004055358FE8003CB
:10302000435801E546D39400400715465358FD80A8
:1030300003435802E4FF74A42FF8E6FEB4021CEF29
:1030400025E02420F582E43401F583E0FCA3E0D3FD
:1030500094F4EC94014004E5578007EEB40108E5D0
:1030600057C313F5578008E557C3134480F5570F2E
:10307000BF08C3E4FFEF25E02430F582E43401F516
:1030800083E0FCA3E0D39400EC9402E559400513DF
:0E309000F5598006C3134480F5590FBF08D7C9
:01309E00220F
:1033570078BEE624FE601A14602A24027038C2B5CB
:10336700C2B6E5486005E4F5808003855780D2B78B
:1033770022C2B7C2B6E5486005E4F58080038558E8
:1033870080D2B522C2B7C2B5E5486005E4F58080B2
:0733970003855980D2B62224
:0436CF00759FA7221A
:0436AA007F507EC30C
:0B36AE00EF1FAC0670011E4C70F622EE
:100D940000C1814001C0804101C0804100C1814047
:100DA40001C0804100C1814000C1814001C0804137
:100DB40001C0804100C1814000C1814001C0804127
:100DC40000C1814001C0804101C0804100C1814017
:100DD40001C0804100C1814000C1814001C0804107
:100DE40000C1814001C0804101C0804100C18140F7
:100DF40000C1814001C0804101C0804100C18140E7
:100E040001C0804100C1814000C1814001C08041D6
:100E140001C0804100C1814000C1814001C08041C6
:100E240000C1814001C0804101C0804100C18140B6
:100E340000C1814001C0804101C0804100C18140A6
:100E440001C0804100C1814000C1814001C0804196
:100E540000C1814001C0804101C0804100C1814086
:100E640001C0804100C1814000C1814001C0804176
:100E740001C0804100C1814000C1814001C0804166
:100E840000C1814001C0804101C0804100C1814056
:100E940000C0C101C30302C2C60607C705C5C40416
:100EA400CC0C0DCD0FCFCE0E0ACACB0BC90908C886
:100EB400D81819D91BDBDA1A1EDEDF1FDD1D1CDC76
:100EC40014D4D515D71716D6D21213D311D1D010E6
:100ED400F03031F133F3F23236F6F737F53534F4D6
:100EE4003CFCFD3DFF3F3EFEFA3A3BFB39F9F83846
:100EF40028E8E929EB2B2AEAEE2E2FEF2DEDEC2C36
:100F0400E42425E527E7E62622E2E323E12120E0A5
:100F1400A06061A163A3A26266A6A767A56564A495
:100F24006CACAD6DAF6F6EAEAA6A6BAB69A9A86805
:100F340078B8B979BB7B7ABABE7E7FBF7DBDBC7CF5
:100F4400B47475B577B7B67672B2B373B17170B065
:100F54005090915193535292965657975595945455
:100F64009C5C5D9D5F9F9E5E5A9A9B5B99595898C5
:100F7400884849894B8B8A4A4E8E8F4F8D4D4C8CB5
:100F84004484854587474686824243834181804025
:103202004100FC08016C00C115C114016500026394
:06321200000A0260000A40
:1032C100C2D8E4786CF6786EF6FB7A00796F7F06E7
:1032D1007EEF120FF208E6FFF46003EF70167B0039
:1032E1007A00796FE4F5347F061231364013786F36
:1032F10076FE8002786FE6FD7C00E4FB7F06120F0C
:0E33010094786FE66003B4FF04786F76FE22C6
:0A36B900C2D8E4786CF6786EF622B1
:0536CA00C213D2D8225A
:03002300022EF9B1
:102EF900C0E0C083C082C0D075D000C000C005C08A
:102F090006309879786CE6C394325007E606247146
:102F1900F8A699C2989000FCE0F562786CE6FD6429
:102F29000770347872E6FE6403600DEEB406028021
:102F390007EEB4100B2016089000FA7408F08044CC
:102F4900EEB4100B7877E624099000FAF0803590FA
:102F590000FA7432F0802D9000FAE0B5050B756225
:102F690000786E7606D216801B786CE6B403157865
:102F790072E6B4190F9000FA7406F08007309904CC
:102F8900C299D213D006D005D000D0D0D082D08338
:032F9900D0E03253
:10354C007873E6FE08E67C002400F527EC3EF526B1
:10355C00AF27FE1224FD50177546051236CA1227E6
:10356C00F7AF27AE26121000AF27AE261213620259
:02357C0036B95E
:0424FD008E288F296D
:102501009000FAE0786C666002C3227871E6FFF40D
:10251100600DEF786F6660077871E66002C322781C
:1025210072E664196002A1ABFB7A0079717D041235
:10253100339E8E2A8F2B7875E6FE08E67C002400F8
:10254100FFEC3EFEEF652B7003EE652A6002C322AD
:102551007874E6FF18E6FEC39F40028002AF06785A
:1025610074E6FDEEC39D400518E6FE8002AE0578D7
:102571006FE6FDC39F4005EDD39E4002C32278A3C1
:10258100E6FF7E0012345B1234247C007D141206B7
:10259100518D2CE4F52DE52DC3952C500B7F647ED8
:1025A100001236AE052D80EED3227872E6FF640369
:1025B100600CEF64066007EF64106002C32278725A
:1025C100E6FF6406703BD3E5299408E528940050A2
:1025D100307874E6FEC39402500990011EE030E0A9
:1025E10020C322EEC39404500990011EE030E11192
:1025F100C3227874E6B4080990011EE030E202C3F8
:1026010022E529640A4528703CEFB4030E123424F4
:102611007C007D051206517870A6057870E664018C
:102621006002C3221234247C007D141206518D2CC9
:10263100E4F52DE52DC3952C500B7F647E001236F9
:10264100AE052D80EE7B007A0079719000FAE024CE
:10265100FEFD12339E8E2A8F2B9000FAE0FD246F2F
:10266100F8E6FE74702DF8E67C002400FFEC3EFED7
:0B267100EFB52B06EEB52A02D322C302
:01267C00223B
:041362008E288F2919
:10136600E4F52EC20C7872E6FFB4061DE4F52E7481
:1013760071252EF8E6F599C2133013FD1236CF0506
:101386002EE52EC3940840E722EF64036002A1EE27
:101396007876E6F52C7871E6F52DF599121FE67844
:1013A60072E6F52D3013FD121FE3E52C25E0F52D31
:1013B6003013FD121FE3E52EC3952C4002A1D17E0A
:1013C60000E529252EFFEE3528FEC3EF9464EE9442
:1013D60000505DE52E2529FF7B007A00792AE4F589
:1013E60033122D964005E4F52AF52B7E00E52925D6
:1013F6002EFFEE3528FEC3EF946EEE94004005E412
:10140600F52D8004E52AF52D3013FD121FE37E002D
:10141600E529252EFFEE3528FEC3EF946EEE9400E7
:101426004005752D018004E52BF52D3013FDA1CA6D
:101436007E00E529252EFFEE3528FEEF64634E700B
:1014460013F52D3013FD121FE390011EE0F52D302C
:1014560013FDA1CAAF2E7E00E529252ECFEE352835
:10146600CF249CCF34FFFED3EF9407EE9400504A6E
:101476007E00E529252EFFEE3528FEEF25E0FFEE5E
:1014860033FE74582FF58274003EF583E0F52D3057
:1014960013FD121FE37E00E529252EFFEE3528FEFB
:1014A600EF25E0FFEE33FE74582FF58274003EF50B
:1014B60083A3E0F52D3013FDA1CA7E00E529252E74
:1014C600FFEE3528FEEF249CFDEE34FFFCD3ED94B1
:1014D6000FEC9400503FEF25E0FFEE33FE74382FFB
:1014E600F58274FF3EF583E0F52D3013FD121FE300
:1014F6007E00E529252EFFEE3528FEEF25E0FFEEDE
:1015060033FE74382FF58274FF3EF583A3E0F52D84
:101516003013FDA1CAAF2E7E00E529252ECFEE356C
:1015260028CF249CCF34FFFEC3EF9412EE940050D4
:101536004A7E00E529252EFFEE3528FEEF25E0FF41
:10154600EE33FE74582FF58274003EF583E0F52DD8
:101556003013FD121FE37E00E529252EFFEE352808
:10156600FEEF25E0FFEE33FE74582FF58274003E41
:10157600F583A3E0F52D3013FD8049AF2E7E00E5FF
:1015860029252ECFEE3528CF249CCF34FFFEC3EF7E
:10159600941AEE9400501EE4F52D3013FD121FE34D
:1015A600E52E2529241CF582E43400F583E0F52D8B
:1015B6003013FD800FE4F52D3013FD121FE3752D5A
:1015C600013013FD121FE3052E61BCC20C3013FD62
:1015D600786BE6F599C2133013FD786DE6F599C27E
:1015E60013301302C18680F97872E664107038F5FC
:1015F6002E7471252EF8E6F52DF599C2133013FDDC
:10160600AF2D121FEA1236CF052EE52EC3940640E3
:10161600E0786BE6F599C2133013FD786DE6F5991F
:10162600C21320135B80FB7872E66419705218E6C9
:10163600F52DF599C2133013FDAF2D121FEA1236A0
:10164600CF7872E6F52DF599C2133013FDAF2D1242
:101656001FEA1236CF786FE6F52DF599C2133013CF
:10166600FDAF2D121FEA1236CF786BE6F599C2133D
:101676003013FD786DE6F599C2133013FD1236CF9F
:011686002241
:041000008E288F297E
:10100400752E01E4F52F7872E66406600241A3C3ED
:10101400E5299464E5289400400221D27874E6948A
:101024000150217876E6FD7C00E4FBFF120F9478F2
:1010340075E6FD7C00E4FB7F01120F9490011EE035
:10104400440180287874E6D39403502A7876E6FD28
:101054007C00E4FB7F02120F947875E6FD7C00E4CB
:10106400FB7F03120F9490011EE04402F0FD7C000C
:10107400E4FB7F6341787874E66408702E08E6FE2A
:1010840008E67C002400FDEC3EFCE4FB7F08120F24
:101094009490011EE04404F0FD7C00E4FB7F6312A5
:1010A4000F947876E690011FF0611A7874E6B4091B
:1010B4001B08E6FE08E67C002400FDEC3EFCE4FB95
:1010C4007F09120F947876E6F51C611A7874E6FFAE
:1010D400B4060A7876E6FD7C00E4FB807B7874E64F
:1010E400FFB40D1FC00708E6FE08E67C002400FDDF
:1010F400EC3EFCD007E4FB120F947876E690017581
:10110400F0611A7874E6FFB40C1B7876E6FD7C0077
:10111400E4FB120F947876E6900177F06002611A8E
:10112400754801611A7874E6FFB410127876E6FD0A
:101134007C00E4FB120F947876E6F52E611A78743D
:10114400E6640A70277870E664016002611A7876B2
:10115400E6FD7C00E4FB7F06120F947876E6786F58
:10116400F67D067CEFE4FF1235B9611AE529640FB8
:10117400452870197874E6FF7876E6FD7C00E4FB78
:10118400120F947876E6B40102801F8028E5296462
:10119400144528702B7874E6FF7876E6FD7C00E42D
:1011A400FB120F947876E6B4010B7587809000FCEF
:1011B4007403F0611AE4F5879000FC7406F0611A78
:1011C4007874E6FF7876E6FD7C00E4FB4178C3E5BD
:1011D40029942CE52894014002611A7873E6FE08EC
:1011E400E67C002400FFEC3ECF249CF529EF34FF7D
:1011F400F528C3E5299412E5289400503808E6FE42
:1012040008E62400F52BEC3EF52AD3E52B94FFE504
:101214002A648094834002611AE52925E0FFE528C9
:1012240033FE74202FF58274013EF583E52AF0A382
:10123400E52BF0611AC3E529941AE5289400503986
:10124400E52924EEF52D7876E6FFC3940640026185
:101254001A7492252DF582E43400F583EFF0E52D20
:10126400244EFF7492252DF582E43400F583E0FDCD
:101274007C00E4FB120F94611AE52964634528603D
:1012840002611A7876E6752A00F52BE4FBAD2BACE7
:101294002A7F63120F947876E690011EF0807778A7
:1012A40072E6641070707876E6F97873E6FE08E604
:1012B4007C002400F529EC3EF528749C2529F529A9
:1012C40074FF3528F528E4FDE9FFC3ED9FEC940095
:1012D40050441236CFAF05EF25E0FB2478F8E6FE44
:1012E40074792BF8E67A002400F52BEA3EF52AE51A
:1012F400292DFFE5283CFEEF25E0FFEE33FE7420A8
:101304002FF58274013EF583E52AF0A3E52BF00D59
:10131400BD00010C80B2E52E647F70357F771236F4
:1013240018E4F52C7B007A00792DE4F534AF2C1207
:101334003136500DE4252CFDE434EEFCAF2D12358E
:10134400B9052CE52CD3941040DAC2AF759F808088
:0D135400FEE52EB4FF07C2AF759F8080FE3E
:011361002269
:0927F700786D76FF786B76FF2205
:071FE300852D99C213AF2DFB
:101FEA00786BE66FFF900D9493786D66796BF7EFD7
:051FFA00900E9493F627
:011FFF0022BF
:08339E008B2E8A2F89308D313E
:1033A6007532007533FF7DFFAF311531EF6026AB07
:1033B6002E0530E530AA2F7002052F14F91205E705
:1033C6006533FF900D94936D753200F533EF900ED3
:0A33D6009493FD80D3E533FEEDFF74
:0133E00022CA
:02364E0000007A
:0732180041005108011C00F8
:1034DF00E4F526751C01D20C7F08122CBD50037524
:1034EF002601751C02122E4D5003752602751C0302
:1034FF001233E1EFD3940040028F2685261CE51C82
:0A350F00FD7C00E4FB7F09020F942D
:102E4D00122F9C900051E0FF139290EFA2E192910E
:102E5D00A2E292927FB11235D712324DEF4E60023F
:102E6D0080287F017E001236AE1233158E1A8F1B0D
:102E7D0012357E400280137F017E001236AE123372
:102E8D00158E278F2812357E40051236C3C3227F3B
:102E9D00017E001236AE1233158E298F2A1236C3DB
:102EAD00E51B2528FFE51A35275403F52B8F2C90AC
:102EBD000051E0B4080EE52AB52C20E529B52B1BF1
:102ECD007D0F8010E52AB52C12E529B52B0D90004C
:102EDD0051E014FDAF28AE27122379900051E00484
:0B2EED00F0E0D3940F40037408F0D312
:012EF80022B7
:1033E100122F9C7FB91235D712324DEF4E60061263
:1033F10036C37F00227F017E001236AE1233158F55
:103401002712357E7F017E001236AE1233158F28CA
:10341100E52762281236C3E52870028003E4F52708
:02342100AF27D3
:013423002286
:102FEC00E51D6FFF900D9493651EF51DEF900E94EB
:032FFC0093F51E2C
:012FFF0022AF
:102A8700751DFF751EFF122F9C7FB71235D71232A7
:102A97004DEF4E600280187F017E001236AE900027
:102AA70051E024F8FF1235D712324DEF4E60030282
:102AB70036C37F017E001236AE1233158F161235DC
:102AC7007E7F017E001236AE8516271233158F17CB
:102AD70012357E7F017E001236AEE517622712336C
:102AE700158F1812357E7F017E001236AEE518620B
:102AF700271233158F1912357E7F017E001236AEED
:102B0700E5196227123315AD07900051E024F8FF4D
:102B1700E434FFFEEF25E0FFEE33FE74002FF5826D
:102B270074003EF583EDF012357E7F017E0012368C
:102B3700AE900051E024F8FFE434FFFEEF25E0FFFC
:102B4700EE33FE74002FF582740012330FAD079039
:102B57000051E024F8FFE434FFFEEF25E0FFEE33F9
:102B6700FE74012FF58274003EF583EDF012357E79
:102B77007F017E001236AE900051E024F8FFE43466
:102B8700FFFEEF25E0FFEE33FE74012FF5827400A0
:102B970012330FEF62271236C3900051E004F0E0C2
:082BA700D3940F40037408F001
:012BAF002203
:022CBD008F275F
:102CBF0078287C007D007BFF7A36794E7E007F146A
:102CCF001205C1C290C291C292122F9C300C047F88
:102CDF00B18005200C057FB21235D77F017E00121F
:102CEF0036AE12324DEF4E600280167F017E00121B
:102CFF0036AE1233158E288F29753C0112357E4062
:102D0F00051236C3C3227F017E001236AEE53C1397
:102D1F009290E53CA2E19291A2E29292123315E5D4
:102D2F003C25E02428F8A60608A607053CE53CD379
:102D3F00940940C81236C3E529252BCFE528352A3B
:102D4F00CF252DCF352CCF252FCF352ECF2531CFDA
:102D5F003530CF2533CF3532CF2535CF3534CF254D
:102D6F0037CF3536CF2539CF35385403FEE53BB550
:102D7F000713E53AB5060E7B007A007928852741BF
:062D8F007D081221CBD3E8
:012D9500221B
:102F9C00C2D97F017E001236AED2DAD2D97F027E40
:102FAC00001236AEC2DA7F057E001236AEC2D97F71
:102FBC00027E001236AEE51CB402028005E51CB49C
:102FCC00031DD2DAD2D97F027E001236AEC2DA7F6E
:102FDC00057E001236AEC2D97F027E001236AE22BA
:10357E00E4FFFE20DA0D0FBF00010EEF64644E7003
:10358E00F2C322D2DA7F017E001236AED2D9C2DA6F
:0C359E007F017E001236AED2DAC2D9D313
:0135AA0022FE
:0235D700AD073E
:1035D9007B08ED3392DAD2D97F017E001236AEC272
:0E35E900D97F017E001236AEED25E0FDDBE459
:0135F70022B1
:06330F003EF583E0622799
:10331500E4FBFAE51CB403047D0880027D0AE4F9A8
:10332500E9C39D5028D2D97F017E001236AED2DA8C
:10333500EB25E0FFEA33FEA2DAE433FBEEFAEF4BCE
:10334500FBC2D97F017E001236AE0980D3AE02AF33
:013355000374
:013356002254
:0736C300C2DAD2D9D2DA22EB
:10324D00E4F53DF53EE51C64017018D2DAD2D9FAE9
:10325D00FB20DA0280460BBB00010AEB640A4A70C0
:10326D00F0804AE51C6402701DFAFB20DA0BD2D9FE
:10327D007F017E001236AE80230BBB00010AEB648A
:10328D00324A70E78027E51C64037027FAFBD2DA17
:10329D0020DA0FD2D97F017E001236AEC2D9E4FEFC
:1032AD00FF220BBB00010AEB64324A70E1C2D97EEA
:0332BD00007F018E
:0132C00022EB
:062379008E2D8F2E8D2F2A
:10237F00E52F25E02420F582E43401F583E0FEA368
:10238F00E0FFC3E52E9FFFE52D9EFE123698D3EF9B
:10239F009464EE6480948040467472252FF582E435
:1023AF003400F583E004F07472252FF582E43400D5
:1023BF00F583E0D364809482500281667472252F76
:1023CF00F582E43400F583E4F0E52F25E02420F5D1
:1023DF0082E43401F583E52DF0A3E52EF0807874C7
:1023EF0072252FF582E43400F583E4F0E52F25E024
:1023FF002420F582E43401F583E0FEA3E0FFE4FC42
:10240F00FD7B02FAF9F8120757C004C005C006C0D9
:10241F0007AE2DAF2EE4FCFD7B08FAF9F812075733
:10242F00D003D002D001D000EB2FFFEA3EFEE93DF2
:10243F00FDE83CFCE47B0AFAF9F81207E28F338ED1
:10244F00328D318C30E52F25E02420F582E43401E4
:10245F00F583EEF0A3EFF0E52F25E02420F582E4DD
:10246F003401F583E0FCA3E0FD748A252FF582E4A7
:10247F003400F583E0FF7B807A0012267DE52F255F
:10248F00E02400F582E43400F583EEF0A3EFF0E5ED
:10249F002F25E02420F582E43401F583E0FEA3E04C
:1024AF00D39400EE94044013E52F25E02420F58209
:1024BF00E43401F5837404F0A3E4F0E52F25E02460
:1024CF0020F582E43401F583E0FEA3E0FFE4FCFD98
:1024DF007B607AEAF9F8C31208825011E52F25E0E4
:0D24EF002420F582E43401F583E4F0A3F02D
:0124FC0022BD
:0821CB008B3D8A3E893F8D40E7
:1021D300E4F544E544C3954040026178AB3DAA3E33
:1021E300A93FE5440475F002A4F58285F083120645
:1021F300C8FFAEF0E544254125E02420F582E43410
:1022030001F583E0FCA3E0FDC3EF9DF543EE9CF5F0
:1022130042C3E5439464E54264809480500DC3E572
:1022230043949CE5426480947F5023E5442541FD1B
:1022330025E02420F582E43401F583EEF0A3EFF0EA
:1022430074722DF582E43400F583E4F08059AB3DDC
:10225300AA3EA93FE5440475F002A4F58285F08304
:102263001206C8FFAEF0E5442541FD25E02420F524
:1022730082E43401F583E0FAA3E0FBC39FEA9E50B6
:102283000F74722DF582E43400F583E004F08017B7
:10229300D3EB9FEA9E4010E54425412472F582E486
:1022A3003400F583E014F0E54425412472F582E41B
:1022B3003400F583E0FFD36480948A500AC3EF644B
:1022C30080947640026174D3E5439414E5426480BC
:1022D3009480500DC3E54394ECE5426480947F50B1
:1022E3001FAE42AF437C007D05120651E5442541F4
:1022F30025E02420F582E43401F583EE8FF0805F3E
:10230300AB3DAA3EA93FE5440475F002A4F58285DE
:10231300F0831206C8FFAEF0E5442541FD25E02415
:1023230020F582E43401F583E0FAA3E0FBC39FEADE
:102333009E5012ED25E02420F582E43401F583E478
:1023430075F001801AD3EB9FEA9E4016E5442541C0
:1023530025E02420F582E43401F58374FFF5F012BF
:102363000687E54425412472F582E43400F583E4CD
:05237300F0054421D635
:012378002242
:103519000205050506060606070707080809090A38
:103529000B0C0C0D0E10121315171B1E252A2F3606
:103539003A3B37312C26231E1D1818151513111166
:03354900100F0F51
:10321F0041019A0041019700016A00C117420198CC
:02322F00012C70
:1008ED00E4F528F529200A3DD293A29033FDA2917B
:1008FD00E433FBA292E433FA90019AE0FF13929055
:10090D00EFA2E19291A2E29292C2B27FF47E011225
:10091D0036AED2B2ED24FF9290EB24FF9291EA24F1
:10092D00FF9292C29390019AE0045407F0900177E0
:10093D00E0FF6002413D300A66200202413D900118
:10094D0097E0640C7057E56A045407F56AC202D249
:10095D000830172625E02420F582E43401F5837450
:10096D0003F0A374E8F0E56AB40702C217E490013E
:10097D0097F0E548602715484137E56A25E02420C2
:10098D00F582E43401F583E4F0A3F0E56AB40702DF
:10099D00D217E4900197F0E54860021548413720E1
:1009AD000202413D90019AE0FE90019830E012E084
:1009BD00FCA3E0FDC374E89DF52774039CF5268028
:1009CD0007E0F526A3E0F527C374079E25E0242054
:1009DD00F582E43401F583E526F0A3E527F09001D7
:1009ED0097E064207044C202D20830171B90019921
:1009FD00E02464F0900198E03400F0E0B40320A30B
:100A0D00E0B4E81BC2178017900199E0249CF09088
:100A1D000198E034FFF0E07002A3E07002D217E419
:100A2D00900197F0E54860021548900197E004F0B9
:100A3D00200A02A12E90019AE0FEB408004002A106
:100A4D0093900A5425E073416441B86112616C6161
:100A5D00C68120817A81D474A42EF8E6FE700CEF45
:100A6D006009300003C2A022D2A022EEB4010F9083
:100A7D000177E06009300003D2A022C2A0229001CC
:100A8D009AE025E02420F582E43401F583E0FEA30D
:100A9D00E0D394F4EE94014009300003D2A022C2B9
:100AAD00A022300003C2A022D2A02290019AE024FD
:100ABD00A4F8E6FF700F900177E06009300003C2E3
:100ACD00A122D2A122EFB4010F900177E06009308D
:100ADD000003D2A122C2A12290019AE025E0242098
:100AED00F582E43401F583E0FEA3E0D394F4EE94B3
:100AFD00014009300003D2A122C2A122300003C25D
:100B0D00A122D2A12290019AE024A4F8E6FF700F51
:100B1D00900177E06009300003C2A222D2A222EF39
:100B2D00B4010F900177E06009300003D2A222C218
:100B3D00A22290019AE025E02420F582E43401F50B
:100B4D0083E0FEA3E0D394F4EE940140093000035A
:100B5D00D2A222C2A222300003C2A222D2A222908D
:100B6D00019AE024A4F8E6FF700F900177E0600988
:100B7D00300003C2A322D2A322EFB4010F9001775C
:100B8D00E06009300003D2A322C2A32290019AE0B3
:100B9D0025E02420F582E43401F583E0FEA3E0D3C3
:100BAD0094F4EE94014009300003D2A322C2A32293
:100BBD00300003C2A322D2A32290019AE024A4F80C
:100BCD00E6FF700F900177E06009300003C2A422A8
:100BDD00D2A422EFB4010F900177E0600930000339
:100BED00D2A422C2A42290019AE025E02420F5820D
:100BFD00E43401F583E0FEA3E0D394F4EE940140D8
:100C0D0009300003D2A422C2A422300003C2A422C0
:100C1D00D2A42290019AE024A4F8E6FF700F90016F
:100C2D0077E06009300003C2A522D2A522EFB401FE
:100C3D000F900177E06009300003D2A522C2A522F2
:100C4D0090019AE025E02420F582E43401F583E05B
:100C5D00FEA3E0D394F4EE94014009300003D2A535
:100C6D0022C2A522300003C2A522D2A52290019A4C
:100C7D00E024A4F8E6FF700F900177E060093000E2
:100C8D0003C2A622D2A622EFB4010F900177E06035
:100C9D0009300003D2A622C2A62290019AE025E0D7
:100CAD002420F582E43401F583E0FEA3E0D394F42F
:100CBD00EE94014009300003D2A622C2A6223000D4
:100CCD0003C2A622D2A62290019AE024A4F8E6FF40
:100CDD00700F900177E06009300003C2A722D2A700
:100CED0022EFB4010F900177E06009300003D2A725
:100CFD0022C2A72290019AE025E02420F582E43457
:100D0D0001F583E0FEA3E0D394F4EE9401400930A5
:100D1D000003D2A722C2A722300003C2A722D2A766
:100D2D002290019AE0FFC374079F24A4F8E6FF7098
:100D3D000A900177E06004E4F5A722EFB4010C906E
:100D4D000177E060067FFF7E03803690019AE0FF19
:100D5D00C374079F25E02420F582E43401F583E078
:100D6D00FEA3E0FF900175E0FD7C00EF2DFFEC3E52
:100D7D00CF2480CF34FFFEC3648094805003E4FE03
:060D8D00FF12309F8FA74A
:010D9300223D
:04309F008E2A8F2BBB
:1030A300E4F52C90351993752D00F52ED3E52E9567
:1030B3002BE52D952A4004E4FFFE22052CAF2CEFCF
:1030C3003395E0FE74192FF58274353EF583E4934E
:1030D300F9252EF52EE4352DF52DD3E52E952BE58B
:1030E3002D952A4046E52E952BFFE52D952AFEE9E1
:1030F300C39FFBE49E7C007D0AAF03FE12063FE9FB
:10310300FD1206517C007D0512063F7D0A12065111
:10311300AA06AB07AF2CEF3395E0FE7C007D0512CA
:10312300063FEF2BFBEE3AAF03FE22E52C708C7FBC
:02313300FFFE9D
:013135002277
:0301000015000DDA
:10363400C0D1CEBBA183674F3D2D9B19273D536657
:0A364400717065554333261C1541D3
:02323100C19842
:041687008E348F35D9
:10168B007B0EEB30180E3395E0FE743F240EF58283
:10169B007436800CFF3395E0FE74342FF58274366C
:1016AB003EF583E493FF900195E4F0A3EFF0D39024
:1016BB000196E09535900195E095344004EBFFE100
:1016CB00C51BEBFF3395E0FE301809743F2FF582F5
:1016DB007436800774342FF58274363EF583E493A9
:1016EB00FF900196E02FF0900195E03400F090010F
:1016FB0095E0FEA3E0FFD39535EE95345002E1BDA6
:10170B00EF9535FFEE9534FE7C007D6412063F901D
:10171B000193EEF0A3EFF0900193E0FEA3E0FFEB5B
:10172B00FD3395E0FC301809743F2DF5827436803B
:10173B000774342DF58274363CF583E493FD7C00FD
:10174B00120651900193EEF0A3EFF0C3EB6480947B
:10175B0084EBFF40253395E0FEEF24FCFFEE34FFD6
:10176B00FE7C007D6412063F900194E02FF0900107
:10177B0093E03EF0E0547FF080533395E0FE7C0025
:10178B007D6412063F900194E02FF0900193E03EB0
:10179B00F0E0FEA3E0FFC374909FFF74019EFE90E8
:1017AB000193F0A3EFF0EE4480900193F0A3EFF0E0
:1017BB00801BEB6002C1CCAF03EF3395E0FE7C00E6
:1017CB007D6412063F900193EEF0A3EFF09001932E
:0517DB00E0FEA3E0FFA9
:0117E00022E6
:10267D0090018CEFF0A3ECF0A3EDF0A3EAF0A3EB47
:10268D00F0EF701E90018FE0FEA3E0FF90018EE051
:10269D002FFF90018DE03ECF2480CF34FF9001912C
:1026AD00E1EA90018CE0FF64016005EF6402707C4B
:1026BD0090018DE0FEA3E0FF12168790018AEEF0E7
:1026CD00A3EFF0EE90018A30E712E0547FFEA3E015
:1026DD00FFC3E49FFFE49E9001918008E0FFA3E01B
:1026ED00900191CFF0A3EFF090018CE0B402229015
:1026FD000191E0FEA3E0FF7C007D0912063F7D0500
:10270D00120651EF2440FFEE3401900191F0A3EF3A
:10271D00F090018FE0FEA3E0FF900192E02FFF907B
:10272D000191E03ECF2480CF34FFE1EA90018CE0AF
:10273D00B40328A3E0FCA3E0FDEC1204377B007A80
:10274D00C0797F7844120395E4FBFA79C878421278
:10275D00028C120470900191EEE1EA90018CE0FF81
:10276D0064046005EF6405707890018DE0FCA3E0D2
:10277D00FDEC1204377B007AC0797F784412039503
:10278D00E4FBFA7948784212028C12047090018AA7
:10279D00EEF0A3EFF0D39418EE648094805012A362
:1027AD00E0FFB40504D20C802BEFB40427C20C80DB
:1027BD0023C390018BE0941A90018AE06480948089
:1027CD00401290018CE0FFB40504C20C8006EFB4FA
:1027DD000402D20CA20CE4FF33900191CFF0A3EFD1
:0927ED00F0900191E0FEA3E0FF71
:0127F60022C0
:103233004401860200020048017E006800690066BE
:09324300006744017A0002000258
:0E35AB00853783E493900191FFF0AC39AD3A7F
:1035B900AB07C2AF75F65575F6AA75F65543BF0444
:0E35C9008CF48DF58BF675F780D2AF7F002263
:10361800C2AF75F65575F6AA75F65543BF04EF2582
:0C362800E0F5F4E4F5F575F782D2AF226E
:0B0FF2008F828E83E49312062D7F0196
:010FFD0022D1
:0C35F800E52775F002A4240CF9E4FAFBAE
:1036040012069DF58285F083E4932402FFE4338F50
:04361400F0020700B9
:02346500A907B5
:10346700E925E0247AF582E43401F583A3E0F53613
:10347700E925E0240CF8E6FE08E6FFE5362402FD20
:10348700E433FCE925E02410F8E6FA08E6C39DFDDD
:0D349700EA9CFCC3EF9DEE9C4002D322C3D3
:0134A4002205
:10368600E4F526AF26121D170526E526C39402404B
:01369600F241
:013697002210
:021D17008F2714
:101D1900EF25E02486F582E43401F583E0F52AA372
:101D2900E0F52BEF25E025E0247EF582E43401F58A
:101D390083A3E0F528EF25E025E02480F582E4344B
:101D490001F583A3E0F529E52825E0F52C752D009B
:101D5900E52925E0752EFFF52F753000852D828543
:101D69002C83E49364556002C1BDAB2EAA2FA93020
:101D79001205E764556002C1BDE52D2401FFE43574
:101D89002CFEE52725E0240CF8A60608A607E5277A
:101D990025E0240CF8E6FE08E6F5828E83E493F448
:101DA9006020E52725E0240CF8E6FE08E6AA06C32C
:101DB900852F838530829582EA958350051235F8FF
:101DC90080CCE52725E0240CF8E6FE08E6C3952D2E
:101DD900F532EE952CF531E5302401F9E4352FFE85
:101DE900AF01E52725E0240CF8A60608A607E52794
:101DF90025E0240CF8E6FE08E6F5828E83E493F4E8
:101E09006030AB2EE530252BF9E52F352AFAC003D2
:101E19008A838982E52725E0240CF8E6FE08E6AAEC
:101E290006F9C3D0E0E99582EA958350051235F8A1
:101E390080BCE52725E0240CF8E6FE08E6AB2EAACF
:101E49002FA930AC02AD01C39DFFEE9CFED3EF95E7
:101E590032EE95315032AE02AF01EF2401FFE43E7C
:101E6900FEE52725E02408F8A60608A60774142528
:101E790027F8A628AE2CAF2DAD07AC06E4FF123526
:101E8900B9EF7002E13EC322E52D2401FFE4352CB0
:101E9900FEE52725E02408F8A60608A607741425F8
:101EA90027F8A629AC2FAD30E4FF1235B9EF70023F
:101EB900E13EC322852D82852C83E493B4551EE52A
:101EC9002D2401FFE4352CFEE52725E02408F8A69A
:101ED9000608A60774142527F8A6298058AB2EAA48
:101EE9002FA9301205E7B45520AE02AF01EF240146
:101EF900FFE43EFEE52725E02408F8A60608A60724
:101F090074142527F8A628802CAE2CAF2DAD07AC6C
:101F190006ED2401FFE43CFEE52725E02408F8A6A8
:101F29000608A60774142527F8A6297F551235B97E
:101F3900EF6002C322E52725E02408F8E6FE08E65B
:101F4900FFE52725E0240CF8A60608A607E52725BE
:101F5900E02408F8E6FE08E6252BFFE52A3EFEE523
:101F69002725E02410F8A60608A607E52725E0247A
:101F79000CF8E6FE08E6F5828E83E493F460051218
:051F890035F880E7D3EC
:011F8E002230
:022000008F3619
:10200200EF25E02408F8E6FE08E68E37F53874146A
:102012002FF8E625E0F539753A00E53625E0248605
:10202200F582E43401F583E0FFA3E0900192CFF062
:10203200A3EFF0E490018EF0E53625E02486F582E8
:10204200E43401F583E0C313FF90018EE0C39FE403
:10205200940050151236CF74142536F8E6FFE02F9F
:10206200FF123618E004F080CF900193E02538FF8C
:10207200900192E03537CF24FFF53CEF34FFF53B7A
:10208200053AE53A70020539853882853783E4934B
:10209200F470022130C3E538953CE537953B4002A8
:1020A20021301236CF853882853783740193FF60E1
:1020B20072F4606FE49390018F1235B3EF60037F87
:1020C2000122053AE53A700205390538E538700211
:1020D2000537F5821235ABEF60037F0122053AE541
:1020E2003A700205390538E53870020537E4900187
:1020F2008EF090018FE0FF90018EE0C39F508985A2
:1021020038821235ABEF60037F0122053AE53A705F
:102112000205390538E5387002053790018EE00472
:10212200F080CF7B007A007937123604018AE536D7
:1021320025E0240CF8A63908A63AE53625E024085D
:10214200F8E6FEEEC313900190F0FD74142536F804
:10215200E625E0FEE53625E02408F8A60608760026
:1021620074142536F8A605E53625E02408F8E6FEBF
:1021720008E6FF900193E02FFF900192E03EFEE51A
:102182003625E02410F8A60608A607E53625E02441
:1021920008F8E6FC08E6FD7F551235B9EF60037FCB
:1021A200012274142536F8E67D0025E0FCE4FF12D6
:1021B20035B9EF60037F0122E53625E02408F808EF
:0821C20006E6187001067F001B
:0121CA0022F2
:082948008F368B378A3889397C
:10295000E4F53EF53FE53A25E0247AF582E43401DA
:10296000F583A3E0F540E53A25E02408F8E6FE0803
:10297000E68E3BF53C0536E53A25E0240CF8E6FE0C
:1029800008E6FFE5402401FDE433FCE53A25E024B8
:1029900010F8E6FA08E6C39DFDEA9CFCD3EF9DEE35
:1029A0009C400122853C82853B83740193FE653601
:1029B0006010E493F4600B7B007A00793B123604DC
:1029C00080E2EEB5360BE53C2401F53FE4353BF5FE
:1029D0003EE53A25E0240CF8E6FE08E6FDAC06AF3D
:1029E000401235B9EF6002C322E53A25E0240CF825
:1029F00008740226F618E436F6E4F53DE53DC39585
:102A0000405030E53A25E0240CF8E6FE08E6253D86
:102A1000FFE43EFEAD07FCAB37AA38A939853D82FD
:102A2000758300120600FF1235B9EF6002C322055C
:102A30003D80C9AF407E00E53A25E0240CF808EF60
:102A400026F618EE36F6E53A25E0240CF8E6FC0802
:102A5000E6FDEF2401FFEE33FEC3ED9FFFEC9EFE8B
:102A6000AD07FCAF361235B9EF6002C322E53F4532
:102A70003E6012AE3EAF3FAD07AC06E4FF1235B983
:062A8000EF6002C322D347
:012A8600222D
:082D96008F2F8B308A31893246
:102D9E00E53325E02408F8E6FE08E68E34F535E442
:102DAE00F536F537052F853582853483E493F46047
:102DBE0049E53325E02410F8E6FC08E6FDC3E535C9
:102DCE009DE5349C5034740193652F7022E5374590
:102DDE00366016E5372401FFE43536FEAD07FCE418
:102DEE00FF1235B9EF6002C3228534368535377B45
:102DFE00007A00793412360480ACE5374536603DF2
:102E0E00853782853683740293FFAB30AA31A9329F
:102E1E00E48FF0120738AB30AA31A93212069D7535
:102E2E00F000120738853782853683740393FFAB23
:0E2E3E0030AA31A932E48FF0120700D322C36C
:012E4C002263
:083136008F308B318A3289339E
:10313E00E53425E02408F8E6FE08E68E35F536E49B
:10314E00F537F5380530853682853583E493F4609E
:10315E0049E53425E02410F8E6FC08E6FDC3E53623
:10316E009DE5359C503474019365307022E53845E9
:10317E00376016E5382401FFE43537FEAD07FCE471
:10318E00FF1235B9EF6002C3228535378536387B9D
:10319E00007A00793512360480ACE5384537601474
:1031AE00853882853783740393AB31AA32A93312E3
:0531BE00062DD322C321
:0131C30022E9
:040F94008F308B31DE
:100F9800E4F532EDF534ECF5331236CFAF311234D7
:100FA800655022E532C3940A500CAF31122000EF8D
:100FB8006004053280ED7F057E001236AEE532C34F
:100FC800940A400122E532C3940A50147B007A0047
:100FD800793385313AAF301229484004053280E52B
:090FE800E532C3940A400122D352
:010FF10022DD
:10028C00EC4D6011E8497017ED33EC3304600DE46C
:10029C00FCFFFEFD22E933E8330470F80204DC12A3
:1002AC0004A758046009E4CC2481500628500902A4
:1002BC0004E62840030204E3C0E0EB4A7044B98032
:1002CC0006D0E0FB0204D2EF4E701CBD8008EBFFA1
:1002DC00EAFEE9FD80EBE98DF0A4FEE5F002037582
:1002EC00E9CDF9EAFEEBFFEF89F0A4FCE5F0CE894D
:1002FC00F0A42EFFE435F0CD89F0A42DFEE435F00A
:10030C008067EF4E7005BD80D780C3EF8BF0A4AC37
:10031C00F0EE8BF0A42CFCE435F0F8EF8AF0A42C72
:10032C00E5F038FCE433CB8DF0A42CFCE5F03BF885
:10033C00EE8AF0A42CFCE5F038F8E433CF89F0A475
:10034C002CFCE5F038CF3400CE89F0A42FFFE5F07B
:10035C003EFEE433C98DF0A42EFEE5F039CD8AF0D3
:10036C00A42FFFE5F03EFEE43DFD33D0E0FB50074B
:10037C000BBB000F0204E6EC2CFCEF33FFEE33FE5C
:06038C00ED33FD0204BE8A
:100392000204E6EC5D046005E8590470030204DC23
:1003A2001204A7580460F6EC4860F2EC7004FDFEFB
:1003B200FF22C860DB2481C85009C398600250063E
:1003C2000204E39850CAF582E9294B4A7005AB82D0
:1003D2000204D275F0007C1A7880C3EF9BEE9AED8E
:1003E20099400DC3EF9BFFEE9AFEED99FDE842F0B6
:1003F200DC23ACF0D0E0FFD0E0FED0E0FDAB822009
:10040200E7101BEB60BAEC2CFCEF33FFEE33FEED92
:1004120033FD0204BEE803F830E705C0F075F000D2
:10042200EF2FFFEE33FEED33FD40B830E7C280AA76
:1004320075F020800E75F010800575F0087D007E45
:10044200007F003392D530D503120874EC3340108C
:10045200EF33FFEE33FEED33FDEC33FCD5F0ED224E
:0E046200E5F0247EA2D513CC92E7CDCEFF228A
:10047000EDD2E7CD33EC3392D524814006E4FFFE84
:10048000FDFC22FCE4CFCECDCC24E0501174FF80E3
:10049000EDC3CC13CCCD13CDCE13CECF13CF047080
:0704A000F030D5DE02087404
:1004A700E9D2E7C933E833F892D5EDD2E7CD33EC9B
:0704B70033FC5002B2D52214
:1004BE00EC30E7100FBF000C0EBE00080DBD00049F
:1004CE000BEB6014A2D5EB13FCED92E7FD2274FF4B
:1004DE00FCFDFEFF22E480F8A2D574FF13FC7D80A4
:0304EE00E480EFB8
:03000000020200F9
:0C020000787FE4F6D8FD7581BE0202474D
:1004F100E709F608DFFA8046E709F208DFFA803EED
:1005010088828C83E709F0A3DFFA8032E309F608D9
:10051100DFFA8078E309F208DFFA807088828C8341
:10052100E309F0A3DFFA806489828A83E0A3F608F5
:10053100DFFA805889828A83E0A3F208DFFA804CCF
:1005410080D280FA80C680D4806980F280338010A6
:1005510080A680EA809A80A880DA80E280CA80330F
:1005610089828A83ECFAE493A3C8C582C8CCC58387
:10057100CCF0A3C8C582C8CCC583CCDFE9DEE78057
:100581000D89828A83E493A3F608DFF9ECFAA9F0D6
:10059100EDFB2289828A83ECFAE0A3C8C582C8CC2C
:1005A100C583CCF0A3C8C582C8CCC583CCDFEADE45
:1005B100E880DB89828A83E493A3F208DFF980CCA7
:1005C10088F0EF60010E4E60C388F0ED2402B404A0
:1005D1000050B9F582EB2402B4040050AF23234547
:0605E10082239005417326
:1005E700BB010689828A83E0225002E722BBFE0212
:0905F700E32289828A83E4932245
:10060000BB010CE58229F582E5833AF583E02250AF
:1006100006E92582F8E622BBFE06E92582F8E222F9
:0D062000E58229F582E5833AF583E4932213
:10062D00BB010689828A83F0225002F722BBFE01AC
:02063D00F322A6
:10063F00EF8DF0A4A8F0CF8CF0A428CE8DF0A42ECF
:02064F00FE2289
:10065100C2D5EC30E709B2D5E4C39DFDE49CFCEEC4
:1006610030E715B2D5E4C39FFFE49EFE120898C39C
:10067100E49DFDE49CFC800312089830D507C3E497
:060681009FFFE49EFE2233
:10068700C5F0F8A3E028F0C5F0F8E58215827002FE
:060697001583E038F0229B
:10069D00BB010A89828A83E0F5F0A3E02250068728
:1006AD00F009E71922BBFE07E3F5F009E3192289EA
:0B06BD00828A83E493F5F0740193221D
:1006C800BB0110E58229F582E5833AF583E0F5F070
:1006D800A3E0225009E92582F886F008E622BBFE4D
:1006E8000AE92582F8E2F5F008E222E5832AF58393
:0806F800E993F5F0A3E9932258
:10070000BB010789828A83020687500B09C5F0273F
:10071000F7C5F01937F722BBFE0D09F8E325F0F312
:10072000C5F019E338F322F889828A83740193258E
:08073000F0C5F0F8E493382253
:10073800BB010A89828A83F0E5F0A3F0225006F70C
:0F07480009A7F01922BBFE06F3E5F009F3192209
:10075700E88FF0A4CC8BF0A42CFCE98EF0A42CFC41
:100767008AF0EDA42CFCEA8EF0A4CDA8F08BF0A4BF
:100777002DCC3825F0FDE98FF0A42CCD35F0FCEB1E
:100787008EF0A4FEA9F0EB8FF0A4CFC5F02ECD39E3
:0F079700FEE43CFCEAA42DCE35F0FDE43CFC2250
:1007A60075F008758200EF2FFFEE33FECD33CDCC0A
:1007B60033CCC58233C5829BED9AEC99E58298408D
:1007C6000CF582EE9BFEED9AFDEC99FC0FD5F0D66A
:1007D600E4CEFBE4CDFAE4CCF9A88222B800C1B994
:1007E6000059BA002DEC8BF084CFCECDFCE5F0CBD2
:1007F600F97818EF2FFFEE33FEED33FDEC33FCEB0B
:1008060033FB10D703994004EB99FB0FD8E5E4F9C5
:10081600FA227818EF2FFFEE33FEED33FDEC33FCB2
:10082600C933C910D7059BE99A4007EC9BFCE99AA6
:10083600F90FD8E0E4C9FAE4CCFB2275F010EF2FEB
:10084600FFEE33FEED33FDCC33CCC833C810D707EB
:100856009BEC9AE899400AED9BFDEC9AFCE899F826
:0E0866000FD5F0DAE4CDFBE4CCFAE4C8F922B9
:0E087400C3E49FFFE49EFEE49DFDE49CFC2295
:10088200EB9FF5F0EA9E42F0E99D42F0EC6480C8ED
:0608920064809845F0228D
:10342400AC66AD67AE68AF69780FEFA2E2EC20E658
:1034340001B35D5E5FF47004FCFDFEFFEF13FFEE6D
:1034440013FEED13FDEC13FCD8E08C668D678E68DB
:103454008F69EE547FFE228E668F67E4F568F56906
:013464002245
:10369800C3EE6480948040028007C3E49FFFE49EE9
:0236A800FE2200
:10020C00022800E493A3F8E493A34003F68001F2E0
:10021C0008DFF48029E493A3F85407240CC8C333F3
:10022C00C4540F4420C8834004F456800146F6DFC2
:10023C00E4800B01020408102040809031C4E47E5D
:10024C00019360BCA3FF543F30E509541FFEE493B7
:10025C00A360010ECF54C025E060A840B8E493A37E
:10026C00FAE493A3F8E493A3C8C582C8CAC583CAA9
:10027C00F0A3C8C582C8CAC583CADFE9DEE780BE61
:01324C000081
:10089800BC000BBE0029EF8DF084FFADF022E4CC44
:1008A800F875F008EF2FFFEE33FEEC33FCEE9DEC0D
:1008B800984005FCEE9DFE0FD5F0E9E4CEFD22ED53
:1008C800F8F5F0EE8420D21CFEADF075F008EF2F9D
:1008D800FFED33FD4007985006D5F0F222C398FD8E
:0508E8000FD5F0EA222B
:00000001FF
